:101000004BC0000064C0000062C0000060C000006F
:101010005EC000005CC000005AC0000058C0000064
:1010200056C0000054C0000052C00000CBC40000F5
:101030004EC000004CC000004AC0000048C0000084
:1010400046C0000044C0000042C0000040C0000094
:101050003EC000003CC000003AC0000038C00000A4
:1010600036C0000034C0000032C0000030C00000B4
:101070002EC000002CC000002AC0000028C00000C4
:1010800026C0000024C0000022C0000020C00000D4
:101090001EC000001CC0000011241FBECFEFD2E014
:1010A000DEBFCDBF11E0A0E0B1E0E4EBFCE102C0A7
:1010B00005900D92A436B107D9F711E0A4E6B1E08E
:1010C00001C01D92A338B107E1F74FD3F1C598CF06
:1010D000982F15C08091F200882371F48091E80068
:1010E0008B7F8093E80003C08EB3882351F08091FA
:1010F000E80082FFF9CF02C08091F100915099235E
:1011000049F7089520917201309171018091700129
:1011100090916F018093690190936A01C901809356
:101120006B0190936C01089580916D01843009F4F6
:101130005AC0853030F4813059F0833009F0C3C093
:101140001FC0853009F4A0C0863009F0BCC0AFC014
:1011500080916E01823008F0B6C0D4DF80916E01BC
:10116000882361F48091690190916A0123E0FC0178
:1011700020935700E89507B600FCFDCF85E008C036
:1011800080916E01882311F0823029F4BBDF89E061
:10119000809301010895813009F095C020E030E08E
:1011A00040E050E0F90184918F3F81F0CA01AA2705
:1011B000BB278093680130936A01209369018AE01C
:1011C0008093010185E08093650108952F5F3F4F73
:1011D0004F4F5F4F2030F0E13F07F0E04F07F0E066
:1011E0005F0701F7089580916E01833051F581E02A
:1011F000809364018091730190917401892B71F047
:1012000080916F01813009F05EC0809172019091F0
:1012100071019093670180936601089580916F0139
:10122000882361F42CE088E190E00FB6F894A8954B
:10123000809360000FBE209360000895109200011B
:101240000895882309F03FC080916F018F3F09F016
:101250003AC0E0E0F0E093E085E090935700E89535
:1012600007B600FCFDCF80935700E89507B600FC59
:10127000FDCFE058FF4F20E1E030F20771F781E148
:1012800080935700E8950895E0916F0180916E0179
:10129000882321F4F0E0EB5FFE4F05C0813099F424
:1012A000F0E0EE52FF4F80818093780108958091A5
:1012B0006E01833041F480916F01882321F4809185
:1012C00070018093680108952F923F924F925F9230
:1012D0006F927F929F92AF92BF92CF92DF92EF92E6
:1012E000FF920F931F93CF93DF9380918101909191
:1012F000820190937401809373018091750188231A
:1013000051F0809175018150809375018091750134
:10131000882309F45D9A80917601882351F08091A9
:10132000760181508093760180917601882309F4BB
:101330005C9A80917C01833009F4B2C1843030F42E
:10134000813071F0823009F0E3C111C1853009F4B8
:10135000C5C1853008F4BAC1863009F0D9C1CDC104
:101360005C9883E0809376018091E800877F80938A
:10137000E80080916401882329F0D6DE5D9A5C9AAA
:10138000109264012091730130917401211531058F
:1013900029F42AC08EB3882309F4BAC18091E800E9
:1013A00082FFF8CF8091F10080936D012150304091
:1013B0003093740120937301EEE6F1E00CC080914C
:1013C000F10081932150304081E0E337F80719F4B0
:1013D0003183208308C08091F200882381F7309305
:1013E000740120937301A0DE80910101853009F022
:1013F000BAC08091730190917401892B21F482E02D
:1014000080930101B0C08AE163DE809169018F7130
:101410005FDEC0916B01D0916C0120916901309128
:101420006A0121968E01021B130B219780916E0198
:10143000882309F093C0180136942794C901A0911C
:101440006801B0E09C01AD0162E0E62EF12C012DB7
:10145000112DE20EF31E041F151F59016A0190E0C1
:1014600099249394B5E0A3E048C08091F2008823CA
:1014700071F48091E8008B7F8093E80004C08EB304
:10148000882309F445C18091E80082FFF8CF0894D1
:10149000210831088091F100682F8091F100782FA8
:1014A000F5010B0190925700E89511249F5F90344D
:1014B00019F021143104A1F4F901B0935700E89513
:1014C00007B600FCFDCF2114310451F0F701A093C1
:1014D0005700E89507B600FCFDCFA801970190E002
:1014E00042E0442E512C612C712CE40CF51C061D9D
:1014F000171DA40CB51CC61CD71C2114310409F0FF
:10150000B4CFD0936A01C093690181E18093570001
:10151000E89527C08091F200882371F48091E8005B
:101520008B7F8093E80004C08EB3882309F4F0C059
:101530008091E80082FFF8CF6091F100809169010D
:1015400090916A01A7D38091690190916A010196F7
:1015500090936A01809369010150104001151105B3
:10156000C9F680E1B5DD8091E8008B7FC3C0809132
:10157000E800877F8093E8005D9883E080937501A1
:1015800004C08EB3882309F4C3C08091E80080FFB3
:10159000F8CF80910101893091F08A3069F480910F
:1015A0006E01813049F48091690190916A018093C4
:1015B000F1009093F1009BC08091780196C06091FA
:1015C0006B0170916C012091690130916A016F5F2C
:1015D0007F4F7B01E21AF30A6150704080916E01E7
:1015E000882389F5870116950795C901A09168019F
:1015F000B0E09C01AD011FC08091F200803271F417
:101600008091E8008E7F8093E80004C08EB3882329
:1016100009F47EC08091E80080FFF8CFF901859140
:1016200094918093F1009093F100015010402E5F4F
:101630003F4F4F4F5F4F01151105F1F670936A014F
:101640006093690129C0823039F523C08091F2008E
:10165000803271F48091E8008E7F8093E80004C0AE
:101660008EB3882309F454C08091E80080FFF8CF3E
:101670000091690110916A01C80104D38093F100BF
:101680000F5F1F4F10936A01009369010894E108EE
:10169000F108E114F104D1F682E08093010127C042
:1016A0008091E800877F8093E800809165018093B6
:1016B000F1001092F1001092F1001092F10080916F
:1016C00001018093F1001092F10011C08091E800B7
:1016D000877F8093E8001092650119C08091E8002F
:1016E000877F8093E800809101018093F1008091D1
:1016F000E8008E7F8093E8000AC08091E800877F31
:101700008093E8005D9A5C9A82E08093010187D023
:10171000DF91CF911F910F91FF90EF90DF90CF90CD
:10172000BF90AF909F907F906F905F904F903F9051
:101730002F9008952BD181E085BF15BE089584B701
:10174000877F84BF88E10FB6F89480936000109281
:1017500060000FBE81E085BF82E085BF8AB18063F3
:101760008AB98BB180638BB90CC1E9DF789401C071
:1017700080D2809100018823D9F780916401882369
:10178000B9F7D8DFE0916601F09167010995FA0198
:10179000923071F0933089F0913029F488E091E033
:1017A00022E130E019C080E090E020E030E014C099
:1017B0008AE191E02BE130E00FC0882339F4809179
:1017C0003501282F30E085E391E006C08091390192
:1017D000282F30E089E391E091838083C901089547
:1017E0008091EB0081608093EB001092ED0060939C
:1017F000EC004093ED008091EE00881F8827881F41
:1018000008951092F4001092F0001092E8001092E7
:10181000ED00EBEEF0E080818E7F80830895809173
:101820007B0188238CF403C08EB38823B1F08091B0
:10183000E80082FFF9CF8091E8008B7F8093E80079
:1018400008958EB3882349F08091E80080FFF9CF96
:101850008091E8008E7F8093E80008959C0140917C
:101860008101509182014617570718F4F90120E0D1
:1018700038C06115710511F0AB01F8CF8091E80017
:101880008E7F8093E80040E050E0F0CF8091E80048
:1018900083FF02C081E008958091E80082FD2DC0A1
:1018A0008EB3882381F18EB3853079F18091E80081
:1018B00080FF17C09091F20006C081918093F100E3
:1018C000415050409F5F4115510511F09032A8F3EF
:1018D00020E0903209F421E08091E8008E7F80932F
:1018E000E8004115510591F6222381F606C08EB31A
:1018F000882349F08EB3853041F08091E80082FF63
:10190000F6CF80E0089582E0089583E0089554D0F2
:1019100056D01EBA1092790184E089BD89B58260E3
:1019200089BD09B400FEFDCF8091D800982F9F7724
:101930009093D80080688093D800809163008E7F58
:10194000809363008091D8008F7D8093D800809130
:10195000E0008E7F8093E0008091E1008E7F809395
:10196000E1008091E20081608093E2008091E100DB
:10197000877F8093E1008091E20088608093E2009D
:101980000895C5DF81E080937A010895C0DFE0EE1D
:10199000F0E0808181608083E8EDF0E080818F77E6
:1019A00080830AD00CD019BCE3E6F0E0808181602E
:1019B000808310927A0108951092E20008951092A7
:1019C000E10008951F920F920FB60F9211242F93EA
:1019D0003F934F935F936F937F938F939F93AF93B7
:1019E000BF93EF93FF938091E10080FF1BC0809134
:1019F000E20080FF17C08091E1008E7F8093E100BC
:101A00008091E2008E7F8093E2008091E20080610D
:101A10008093E2008091D80080628093D80019BC46
:101A20001EBA26D18091E10084FF29C08091E20096
:101A300084FF25C084E089BD89B5826089BD09B471
:101A400000FEFDCF8091D8008F7D8093D8008091DB
:101A5000E1008F7E8093E1008091E2008F7E809391
:101A6000E2008091E20081608093E2008091790140
:101A7000882311F481E001C084E08EBBF9D080910D
:101A8000E10083FF22C08091E20083FF1EC08091AD
:101A9000E100877F8093E10082E08EBB10927901A4
:101AA0008091E1008E7F8093E1008091E2008E7F43
:101AB0008093E2008091E20080618093E200A1DEE9
:101AC00080E060E042E28CDED3D08091E10082FFD2
:101AD0000AC08091E20082FF06C08091E1008B7F06
:101AE0008093E100C5D0FF91EF91BF91AF919F919D
:101AF0008F917F916F915F914F913F912F910F90B7
:101B00000FBE0F901F9018951F93DF93CF9300D0B7
:101B1000CDB7DEB7EBE7F1E08091F100819381E092
:101B2000E338F807C9F790917B0180917C018530FB
:101B300011F1863040F48130B9F0813070F083309B
:101B400009F081C011C0883009F453C0893009F40C
:101B500062C0863009F077C02DC0903809F474C097
:101B6000923809F070C070C0992309F46DC09230AA
:101B700009F069C069C0992309F065C010917D0121
:101B80008091E800877F8093E80049DE04C08EB32F
:101B9000882309F459C08091E80080FFF8CF812F95
:101BA0008F7711F492E001C093E09EBB8068809330
:101BB000E3004AC09058923008F045C080917D0102
:101BC00090917E0160917F01AE014F5F5F4FDFDD3D
:101BD000BC010097C9F18091E800877F8093E800FD
:101BE00089819A813BDE8091E8008B7F8093E800B9
:101BF0002BC0903841F58091E800877F8093E80002
:101C0000809179018093F1008091E8008E7F80932C
:101C1000E80005DE19C09923B1F490917D0192305E
:101C200098F48091E800877F8093E8009093790191
:101C3000F6DD80917901882311F483E001C084E00E
:101C40008EBB16D001C040DB8091E80083FF0AC044
:101C50008091EB0080628093EB008091E800877FA9
:101C60008093E8000F900F90CF91DF911F9108951E
:101C700008958EB3882329F08091E80083FF01C086
:101C800043CF0895F999FECF92BD81BDF89A992767
:101C900080B50895262FF999FECF1FBA92BD81BD58
:101CA00020BD0FB6F894FA9AF99A0FBE01960895DE
:041CB000F894FFCFD6
:101CB40001021E938220DCFB1201100100000020AF
:101CC400EB03F72F00000001000109021B000101D2
:101CD4000080320904000000FE0102000921030013
:101CE40000000C0001040309042803530070006180
:101CF4000072006B00460075006E00200042006F09
:101D0400006F0074006C006F006100640065007275
:041D140000000000CB
:0400000300001000E9
:1000000096C00000AFC00000ADC00000ABC0000053
:10001000A9C00000A7C00000A5C00000A3C0000048
:10002000A1C000009FC000009DC0000054C400009B
:1000300018C4000097C0000095C0000093C00000E5
:1000400091C000008FC000008DC000008BC0000078
:1000500089C0000087C0000085C0000008C1000002
:1000600081C000007FC000007DC000007BC0000098
:1000700079C0000012011001020000084F1B0100AE
:1000800000000102000109023E00020100C0320925
:1000900004000001020201000524000110042402F2
:1000A000060524060001070582030800FF09040174
:1000B00000020A0000000705040210000107058382
:1000C00002100001040309043603530070006100AC
:1000D00072006B00460075006E002000280077005B
:1000E000770077002E0073007000610072006B00D3
:1000F000660075006E002E0063006F006D00290021
:1001000000002A0353007000610072006B0046007B
:1001100075006E00200055005300420074006F000F
:10012000530065007200690061006C00000011243A
:100130001FBECFEFD2E0DEBFCDBF11E0A0E0B1E047
:10014000E4E4FFE002C005900D92A631B107D9F7B3
:1001500012E0A6E1B1E001C01D92AF32B107E1F7B4
:10016000F3D0EEC64DCF9C01DC01AE57BF4FED91F1
:10017000FC91119741911196FC93EE9380589F4FFB
:10018000E817F90711F42D933C939FB7F894F90100
:10019000EC57FF4F8081815080839FBF842F08954B
:1001A000DF92EF92FF920F931F93FC0184898130BD
:1001B00019F0823021F405C040E3D42E04C0DD24C0
:1001C00002C030E2D32E8389823011F488E0D82A2D
:1001D0008589873031F0883031F0863031F482E023
:1001E00003C084E001C086E0D82A1092C9001092B2
:1001F000C8001092CA00E784F0880189128980E063
:10020000E81681EEF80680E0080780E0180719F488
:1002100020E130E00FC0C801B7019695879577952A
:10022000679560587B47814E9F4FA801970166D61E
:10023000215030403093CD002093CC00D092CA00A2
:1002400080E0E81681EEF80680E0080780E01807F5
:1002500011F082E001C080E08093C80088E98093BB
:10026000C9001F910F91FF90EF90DF9008951F92AA
:100270000F920FB60F9211242F938F939F93EF93AA
:10028000FF939091CE008EB38430F1F4E091990108
:10029000F0919A019083E0919901F0919A01CF0138
:1002A000019690939A01809399018959914021F484
:1002B00089E191E0928381839FB7F89480919D01B9
:1002C0008F5F80939D019FBFFF91EF919F918F91D1
:1002D0002F910F900FBE0F901F901895FC018585F0
:1002E00080FF02C05F9808955F9A089580E091E0D2
:1002F0009BC580E091E04EC584B7877F84BF28E12D
:100300000FB6F89420936000109260000FBE87E64D
:1003100090E09093CD008093CC0086E08093CA005B
:100320001092C8002093C900539A5A9A8AB18063E8
:100330008AB98BB180638BB989D284E085BD5F9A1D
:10034000579A209A289A08950F931F93CF93DF937B
:10035000D3DF2FB7F8948EE991E090931F0280933A
:100360001E0290932102809320022FBF2FB7F89492
:1003700089E191E090939A018093990190939C0177
:1003800080939B012FBF7894CEE9D1E003E08FB733
:10039000F894909122028FBF903809F180E091E0AB
:1003A0006FD497FD1CC0E0911E02F0911F02808364
:1003B000E0911E02F0911F02CF01019690931F025F
:1003C00080931E028E51924011F4D283C1839FB755
:1003D000F894809122028F5F809322029FBF8FB793
:1003E000F89410919D018FBFA89902C0113690F129
:1003F000A89A80919D01882369F05D980093160169
:10040000289808C089E191E0AEDE682F80E091E095
:100410009DD411501123B1F780911601882359F012
:1004200080911601815080931601809116018823D6
:1004300011F45D9A289A80911701882359F08091D0
:10044000170181508093170180911701882311F4BF
:100450005C9A289A8FB7F894909122028FBF9923C3
:1004600071F08EE991E07FDE982F8091C80085FFC2
:10047000FCCF9093CE0028985C980093170180E001
:1004800091E055D4EAD383CFDA01923049F093302A
:1004900061F09130F9F4E4E7F0E022E130E01EC0D1
:1004A000E6E8F0E02EE330E019C0813049F0813019
:1004B00018F0823079F408C0E4ECF0E0849107C0D1
:1004C000E8ECF0E0849103C0E2E0F1E08491282FB1
:1004D00030E004C0E0E0F0E020E030E0ED93FC9399
:1004E000C901089528E030E040E003C04F5F220FCB
:1004F000331F28173907D0F3842F8295807F089502
:100500008093E9008091EB0081608093EB00109272
:10051000ED006093EC004093ED008091EE00881FA9
:100520008827881F08951092F40090E09093E900C6
:100530001092F0001092E8001092ED008091EB0014
:100540008E7F8093EB009F5F953081F708958091B7
:10055000270288238CF403C08EB38823B1F08091E6
:10056000E80082FFF9CF8091E8008B778093E80064
:1005700008958EB3882349F08091E80080FFF9CF79
:100580008091E8008E778093E800089594E680914A
:10059000EC0080FF05C08091E80080FF05C023C00B
:1005A0008091E80082FD1FC08EB3882311F482E0A1
:1005B00008958EB3853011F483E008958091EB00A7
:1005C00085FF02C081E008958091E10082FFDFCFC6
:1005D0008091E1008B7F8093E100992311F484E006
:1005E00008959150D4CF80E008959C0140912D0250
:1005F00050912E024617570718F4F90120E038C031
:100600006115710511F0AB01F8CF8091E8008E778C
:100610008093E80040E050E0F0CF8091E80083FF55
:1006200002C081E008958091E80082FD2DC08EB364
:10063000882381F18EB3853079F18091E80080FFC5
:1006400017C09091F20006C081918093F100415053
:1006500050409F5F4115510511F09830A8F320E0FC
:10066000983009F421E08091E8008E778093E800CB
:100670004115510591F6222381F606C08EB38823D9
:1006800049F08EB3853041F08091E80082FFF6CFCB
:1006900080E0089582E0089583E008959C014091F0
:1006A0002D0250912E024617570710F490E03BC0E0
:1006B0006115710511F0AB01F9CF8091E8008E77DB
:1006C0008093E80040E050E0F1CF8091E80083FFA4
:1006D00002C081E008958091E80082FD30C08EB3B1
:1006E000882399F18EB3853091F18091E80080FFE5
:1006F0001AC08091F20009C0F9012F5F3F4FE491C9
:10070000E093F100415050408F5F4115510511F0C9
:10071000883090F390E0883009F491E08091E8000F
:100720008E778093E8004115510579F6992369F693
:1007300006C08EB3882349F08EB3853041F0809196
:10074000E80082FFF6CF80E0089582E0089583E01C
:1007500008959C016115710529F48091E8008B775B
:100760008093E800F90120C08091E80083FF02C077
:1007700081E008958EB3882339F18EB3853031F14D
:100780008091E80082FFF0CF06C08091F100819354
:100790006150704021F08091F2008823B1F7809180
:1007A000E8008B778093E80061157105E9F606C0D3
:1007B0008EB3882349F08EB3853041F08091E800F4
:1007C00080FFF6CF80E0089582E0089583E00895E9
:1007D00042D044D01EBA10922502109224021092E8
:1007E000230284E089BD89B5826089BD09B400FE19
:1007F000FDCF8091D800982F9F779093D800806884
:100800008093D800809163008E7F809363008091F5
:10081000D8008F7D8093D8008091E0008E7F8093F8
:10082000E0008091E1008E7F8093E1008091E20002
:1008300081608093E2008091E100877F8093E100F6
:100840008091E20088608093E2000895C1DF81E03A
:100850008093260208951092E20008951092E1001C
:1008600008951F920F920FB60F9211241F932F938A
:100870003F934F935F936F937F938F939F93AF9328
:10088000BF93EF93FF93E9EEF0E0108117701082B1
:10089000E0EFF0E08081877F80837894C3D0F89484
:1008A000A9EEB0E01C92E0EFF0E0808188608083E8
:1008B0001C93FF91EF91BF91AF919F918F917F9189
:1008C0006F915F914F913F912F911F910F900FBEAC
:1008D0000F901F9018951F920F920FB60F92112430
:1008E0002F933F934F935F936F937F938F939F9338
:1008F000AF93BF93EF93FF938091E10080FF1BC004
:100900008091E20080FF17C08091E1008E7F80938C
:10091000E1008091E2008E7F8093E2008091E2000E
:1009200080618093E2008091D80080628093D8003B
:1009300019BC1EBA91D18091E10084FF29C0809139
:10094000E20084FF25C084E089BD89B5826089BD4D
:1009500009B400FEFDCF8091D8008F7D8093D80030
:100960008091E1008F7E8093E1008091E2008F7E94
:100970008093E2008091E20081608093E2008091A8
:100980002502882311F481E001C084E08EBB64D18C
:100990008091E10083FF27C08091E20083FF23C0A4
:1009A0008091E100877F8093E10082E08EBB10920E
:1009B00025028091E1008E7F8093E1008091E2002A
:1009C0008E7F8093E2008091E20080618093E2005C
:1009D000AADD80E060E042E093DD8091F000886075
:1009E0008093F00039D18091E10082FF0AC08091AC
:1009F000E20082FF06C08091E1008B7F8093E100DE
:100A00002BD1FF91EF91BF91AF919F918F917F91EA
:100A10006F915F914F913F912F910F900FBE0F906B
:100A20001F9018951F93DF93CF9300D0CDB7DEB7FB
:100A3000E7E2F2E08091F100819382E0EF32F80783
:100A4000C9F78091270230912802353009F487C018
:100A5000363040F43130C9F1313070F0333009F0C4
:100A6000E6C033C0383009F4B8C0393009F4C7C023
:100A7000363009F0DCC092C0803821F0823809F0AD
:100A8000D6C008C09091230280912402882399F057
:100A9000926011C080912B0287708093E900809151
:100AA000EB0090E025E0969587952A95E1F7982F41
:100AB00091701092E9008091E800877F8093E800B0
:100AC0009093F1001092F10093C0882319F08230C6
:100AD00009F0ADC090E08F719070009721F00297FF
:100AE00009F0A6C00CC080912902813009F0A0C095
:100AF00010922402333069F5809324022AC0809139
:100B00002902882331F520912B02277009F490C027
:100B10002093E9008091EB0080FF8AC0333021F4FC
:100B20008091EB00806213C08091EB008061809324
:100B3000EB0081E090E002C0880F991F2A95E2F750
:100B40008093EA001092EA008091EB008860809325
:100B5000EB001092E9008091E800877F4CC0882369
:100B600009F065C0109129028091E800877F809389
:100B7000E800EDDC04C08EB3882309F459C08091ED
:100B8000E80080FFF8CF812F8F7711F492E001C049
:100B900093E09EBB80688093E3004AC08058823017
:100BA00008F045C08091290290912A0260912B02A1
:100BB000AE014F5F5F4F68DCBC010097C9F18091C7
:100BC000E800877F8093E80089819A8167DD8091C2
:100BD000E8008B778093E8002BC0803841F5809146
:100BE000E800877F8093E800809125028093F100E0
:100BF0008091E8008E778093E800A9DC19C08823F3
:100C0000B1F490912902923098F48091E800877FA6
:100C10008093E800909325029ADC80912502882336
:100C200011F483E001C084E08EBB63DB01C05EDBB6
:100C30008091E80083FF0AC08091EB00806280937E
:100C4000EB008091E800877F8093E8000F900F9081
:100C5000CF91DF911F91089508951F938EB388233C
:100C600061F01091E9001092E9008091E80083FFA3
:100C700001C0D8DE17701093E9001F910895089500
:100C8000FC018EB3843021F587859089A189B289D2
:100C90000097A105B105E1F085818093E90080917D
:100CA000E80082FF15C08091F200882319F42FEF2D
:100CB0003FEF04C08091F100282F30E08091F200D6
:100CC000882341F48091E8008B778093E80002C08C
:100CD0002FEF3FEFC9010895FC018EB3843011F569
:100CE00087859089A189B2890097A105B105D1F0C6
:100CF00081818093E9008091F2008823A9F090918E
:100D0000E8008091E8008E778093E80095FD0CC0A4
:100D10003DDC982F882349F48091E8008E778093FA
:100D2000E80003C092E001C090E0892F0895FC0123
:100D30008EB3843051F487859089A189B289009758
:100D4000A105B10511F0CF01C7CF08951F93FC0194
:100D5000162F8EB38430D9F487859089A189B28902
:100D60000097A105B10599F081818093E9008091F8
:100D7000E80085FD08C08091E8008E778093E80048
:100D800005DC882329F41093F10080E001C082E0A3
:100D90001F9108950F931F93CF93DF93EC010D964E
:100DA000FC0189E0DF011D928A95E9F72A813B81E8
:100DB00009818C81882311F410E001C014E0C9017D
:100DC00091DB182B1260802F61E8412F99DB88237B
:100DD00029F12E813F810D818885882311F410E04F
:100DE00001C014E0C9017EDB182B1260802F60E87F
:100DF000412F86DB882391F02A853B8509858C85E8
:100E0000882311F410E001C014E0C9016BDB182B3A
:100E10001260802F61EC412F73DB01C080E0DF9115
:100E2000CF911F910F910895CF93DF93EC018091A3
:100E3000E80083FF60C0888190E020912B02309110
:100E40002C022817390709F056C0809128028132F8
:100E500061F0823220F4803209F04DC019C0823234
:100E600069F1833209F047C038C080912702813A86
:100E700009F041C08091E800877F8093E800CE01AF
:100E80000F9667E070E0B1DB8091E8008B7713C0CC
:100E900080912702813279F58091E800877F8093E5
:100EA000E800CE010F9667E070E053DCCE0178D900
:100EB0008091E8008E778093E8001DC08091270222
:100EC0008132C9F48091E800877F8093E8008091A7
:100ED00029028D87CE0102DA0DC08091270281326E
:100EE00051F48091E800877F8093E800CE01609103
:100EF0002902C5DE2CDBDF91CF910895A1E21A2EE5
:100F0000AA1BBB1BFD010DC0AA1FBB1FEE1FFF1FAD
:100F1000A217B307E407F50720F0A21BB30BE40BFD
:100F2000F50B661F771F881F991F1A9469F7609544
:100F30007095809590959B01AC01BD01CF010895FE
:040F4000F894FFCF53
:100F4400000310000004100000020800000000006C
:060F540000000000000097
:00000001FF
